S01100004D61696E626F6172642E7372656386
S11300000C943B000C9463000C9463000C94630008
S11300100C9463000C9463000C9463000C946300D0
S11300200C9463000C9463000C9463000C946300C0
S11300300C9463000C9463000C9463000C946300B0
S11300400C9463000C9463000C9463000C946300A0
S11300500C9463000C9463000C9463000C94630090
S11300600C9463000C9463000C9463000C94630080
S11300700C9463004B0211241FBECFEFD4E0DEBF0B
S1130080CDBF11E0A0E0B1E0EAE1F5E002C00590E7
S11300900D92A630B107D9F721E0A6E0B1E001C086
S11300A01D92A930B207E1F710E0C6E7D0E004C022
S11300B02297FE010E948702C437D107C9F70E9424
S11300C0F9010C948B020C940000CF93DF9300D0C1
S11300D0CDB7DEB76EBD65E0CE0102960E94EF019A
S11300E00DB407FEFDCF60E0CE0101960E94EF0142
S11300F08EB50F900F90DF91CF91089584B18660F3
S113010084B985B1817F85B9249A2C9A089580E5B4
S11301108CBD81E08DBD08950F931F93CF93DF9322
S1130120EC01062F142F2C9862E00E946500602FCA
S1130130CE010E946500612FCE010E9465002C9AB9
S1130140DF91CF911F910F910895CF93DF93EC012D
S11301502C9860EC0E9465008FE99FE00197F1F70D
S113016000C000002C9A8FE39CE90197F1F700C0CE
S1130170000047E06AE2CE010E948C0040E969E297
S1130180CE010E948C0042E068E2CE010E948C0005
S113019043E06BE2CE010E948C0040E660E6CE01B3
S11301A00E948C0040E660E7CE010E948C0040E093
S11301B060E2CE010E948C0040E061E2CE010E9428
S11301C08C0040E062E2CE010E948C0040E063E2D9
S11301D0CE010E948C0040E064E2CE010E948C00BB
S11301E040E065E2CE010E948C0040E066E2CE0170
S11301F00E948C0040E067E2CE010E948C0040E047
S11302006CE0CE010E948C00DF91CF910895CF93D2
S1130210DF93EC018FE39CE90197F1F700C0000044
S1130220CE010E947E00CE010E948700CE010E9472
S1130230A500DF91CF910895FF920F931F93CF9361
S1130240DF93EC01F62E042F122F2C9865E00E9408
S113025065006F2DCE010E946500602FCE010E94C3
S11302606500612FCE010E9465002C9ADF91CF9129
S11302701F910F91FF9008951F93CF93DF93EC018B
S11302802C9860EB0E9465006FEFCE010E94650020
S1130290182F6FEFCE010E9465002C9A812FDF91F9
S11302A0CF911F910895AF92BF92CF92DF92EF92B8
S11302B0FF920F931F93CF93DF931F92CDB7DEB7B7
S11302C07C016B010E943C018983898186FF06C001
S11302D02C9860E9C7010E94650009C089818823C0
S11302E00CF069C02C9864E9C7010E9465006FEFA7
S11302F0C7010E94650090E0880F991F880F991F1D
S1130300880F991FF601918380836FEFC7010E94C4
S1130310650090E096958795929582958F708927D0
S11303209F708927F60120813181822B932B918341
S113033080836FEFC7010E9465006FEFC7010E94C1
S113034065006FEFC7010E9465008F70F60183831B
S11303508823A1F086010C5F1F4F5601F5E0AF0E14
S1130360B11C8150A80EB11C6FEFC7010E9465003B
S1130370F80181938F01EA15FB05B1F72C9A898165
S113038083FF04C081E0F601828302C0F601128279
S1130390898186FF07C020E041E06CE2C7010E942A
S11303A01C0106C020E042E06CE2C7010E941C016F
S11303B08981877001C08FEF0F90DF91CF911F91DA
S11303C00F91FF90EF90DF90CF90BF90AF90089582
S11303D084B1806E84B908950E94E801089585B1BE
S11303E08F7185B985B16295660F607E682B65B99A
S11303F00895CF93DF93CDB7DEB72C970FB6F8945B
S1130400DEBF0FBECDBF66E088E091E00E94EF0141
S113041060E071E087E091E00E94700283E291E085
S11304209A8389831B8282E08C838FEA8D838EEF8B
S11304308E8362E088E091E00E94EF012FEF83ED6C
S113044090E3215080409040E1F700C00000BE01DD
S11304506F5F7F4F86E091E00E9453018F3F61F40C
S113046064E088E091E00E94EF018FE39CE901974A
S1130470F1F700C00000DDCF61E088E091E00E9468
S1130480EF019FEF23ED80E3915020408040E1F79E
S113049000C00000CECF88E091E00E94EC0187E02C
S11304A091E00E946D0286E091E00E9407010895A8
S11304B0E8ECF0E0808185FFFDCF6093CE0080E022
S11304C0089586E08093CA00E9ECF0E080818860BA
S11304D0808387E68093CC0008950E94610208958A
S11304E00F931F93CF93DF938C01EB0168816623F5
S11304F039F02196C8010E94580269916111FACF1E
S1130500DF91CF911F910F910895EE0FFF1F05907A
S10D0510F491E02D0994F894FFCF54
S109051A626C610A00009E
S9030000FC
